:1000000000308A00AD2C0000F93083168600831280
:1000100006110330F700F70B0B2806150034071103
:100020004B0893000330F700F70B14280000000082
:100030004C0893000330F700F70B1C280000000069
:100040004D0893000330F700F70B24280000000050
:1000500050308400130880004E0893000330F700EE
:10006000F70B3028000000004F3084001308800098
:100070000730F700F70B3A280000000007154F087B
:10008000F8005008F9000034F93083168600D230A9
:100090008700223085008801890106309F00810198
:1000A00083129F01071518308500890104209817D5
:1000B0008316990118161813981798161417831297
:1000C00094160230CB000B30CC002030CD00203015
:1000D000CE000F208A110A12B72C4B308400000882
:1000E000031981280130F800F701F70B7528F80B88
:1000F00074284A30F700F70B7B2800000000800BC3
:1001000072280034851E822800348220FF30831636
:1001100088008312880185110808A00085158220B7
:1001200085110808A1008515831688018312003403
:100130008518982805150000000005116430CB00D3
:100140006D2007308900EC308800822005120516EA
:1001500085208A110A12C42C0F30CE05E030CE045F
:100160004E3084000008880006308900051205160C
:100170004D308400000888000530890005120516FE
:100180004C308400000888000430890005120516F0
:100190004B308400000888000330890005120516E2
:1001A00001308800023089000512051620308800D1
:1001B000073089000512051689010034C6080319A5
:1001C000E928822085118515822085118515C603B1
:1001D000DE280034F801F901F701FA014C08031D8B
:1001E000F4284B0803190E291030CD000310C90D57
:1001F000CA0DF70DFA0D4C087A02031D01294B08B0
:100200007702031C0A294B08F702031CFA034C0867
:10021000FA020314F80DF90DCD0BF62800008A112F
:100220000A12B0291030F700FA01CB01C80CC70C34
:10023000031C20294908FA070318CB0A4A08CB07F0
:10024000CB0CFA0CF90CF80CF70B16290034CE0184
:10025000CD01CC01CB01AC20E330C600DE208520EF
:10026000C6012108C500A500A4012008A4070318A1
:10027000A50AC801C7012508C6002408C50048080A
:10028000CE004708CD004608CC004508CB00AC2086
:100290000530C600DE208520BD012108BC00852078
:1002A000C6012008C500FA000030BC070318BD0ACB
:1002B0007A08BD072108A2008520C6012108C500D3
:1002C000C800C70120084707BE004808BF00031840
:1002D000BF0A85202008C400C1012108C000852074
:1002E000C6012008C500FA000030C0070318C10A83
:1002F0007A08C10785208520C6012108C500FA00BB
:1003000000302007C2007A08C3000318C30A400D5A
:10031000C500410DC600C50DC60DC50DC60DC50DE8
:10032000C60DC50DC60DE030C50501303C02F70015
:100330003D08FA000030031C0130FA027708450737
:10034000C7004608C8000318C80A7A08C807480842
:10035000CA004708C9003D08CC003C08CB00EA2889
:100360007908A7007808A600C8014408C700430818
:10037000CA004208C90012217908FA0078083E072D
:10038000C5003F08C6000318C60A7A08C607260833
:100390004507A8004608A9000318A90A2708A907C5
:1003A000C6014408C5004608C8004508C700430800
:1003B000CA004208C90012217908FA0078083E07ED
:1003C000AC003F08AD007A0803187A0FAD07AE0104
:1003D000AF018A110A12C52C871C032ACC01CB015C
:1003E0004C08073C031C032ACD0107144D08990053
:1003F0000000000007100000000000000000CB0A11
:100400000319CC0AF02900340230CB00CC010330B0
:10041000CD000430CE000F200230CB00CC010330E1
:10042000CD00CE010F20EC21003486140830F800F6
:10043000000000000000F8172D2AF813C20C031862
:100440008610031C861478172D2A7813F80B1E2AA1
:1004500000000000000086102D2A1C308400840B50
:100460002F2A0000F81B1D2A781B252A0034203073
:10047000DF00DB01DC01DD01DE015608FA00550872
:10048000F9005408F8005308F7000310771C562AA7
:100490005708DB0758080318580FDC0759080318DA
:1004A000590FDD075A0803185A0FDE07DE0CDD0C62
:1004B000DC0CDB0CFA0CF90CF80CF70CDF0B452A02
:1004C0008A110A125B2B3D0CFA003C0CF900FA0C65
:1004D000F90CFA0CF90CFA0CF90C0F30FA05790842
:1004E0002C07C2002D08C3007A0803187A0FC3072F
:1004F0002E08C400003003180130C4072F08C500BF
:10050000003003180130C50724084207C60043081D
:10051000C70025080318250FC7074408C800003086
:1005200003180130C8074508C9000030031801301E
:10053000C9074908CE004808CD004708CC00460846
:10054000CB00AC203C080F39C2003D080039C30085
:10055000420DC400430DC500C40DC50DC40DC50D2D
:10056000C40DC50DF030C4054408C600DE2085204A
:10057000A008031DBE2A0230F800A42B2008E53C89
:100580000319A22BFE30C20015220130C200152231
:100590002008C20015222108C2001522852020084B
:1005A000C20015222108C200152285202008C200A1
:1005B00015222108C200152285202008C20015221C
:1005C0002108C20015222E30C200152285202008E5
:1005D000C20015222108C20015222008BF002108F0
:1005E000C00085202008C20015222108C200152263
:1005F0002008C1003F086D3C0319022B3F084D3C09
:10060000031DA22B4008503C03190A2B4008703CE4
:10061000031DA22B4108333C031DA22B0730C6004B
:10062000DE208520C501C401C3012008C200C90124
:10063000C801C7012108C6004808FA004708F900A8
:100640004608F800F70177084207CB004308CC00C2
:1006500078080318780FCC074408CD0079080318F0
:10066000790FCD074508CE007A0803187A0FCE0718
:1006700002304B02CF004C08D0000030031C013088
:10068000D0024D08D1000030031C0130D1024E08C9
:10069000D2000030031C0130D2025208D6005108AB
:1006A000D5005008D4004F08D300DA01D901D80191
:1006B0002208D700372A7A08D3007908D2007808B0
:1006C000D1007708D00024085007D4005108D50085
:1006D00025080318250FD5075208D6000030031847
:1006E0000130D6075308D700003003180130D70770
:1006F00028085407B0005508B10029080318290F2D
:10070000B1075608B200003003180130B20757088D
:10071000B300003003180130B30785203430840063
:100720002008800035308400210880008520363084
:1007300084002008800037308400210880000130C8
:10074000F800A42B0030F8000034C901042243084B
:100750004702031CA82C031DBD2B42084602031CA4
:10076000A82C031DBD2B41084502031CA82C031D0A
:10077000BD2B40084402031CA82C4308CE004208AD
:10078000CD004108CC004008CB00AC204D14FF3018
:100790008316880010308312CC00CC080319F12B8B
:1007A0008718D42B4D10D02B1030CB00CB08031959
:1007B000EF2B822085110714080899008515071072
:1007C0000000000000000000000085110714080868
:1007D00099008515071000000000CB03D62BCC0331
:1007E000CD2B83168801003083124D180130F8009C
:1007F000F8080319162CC90A4908783C0318152C67
:100800000330CB000B30CC00CD01CE010F20780897
:10081000B800042004220230CB000B30CC00380892
:10082000CD003808CE000F20C9011D2CC90349088E
:10083000013C031C1D2C0230C9008619622C481093
:10084000FA30CA000330CB000B30CC000330CD00AF
:100850001430CE000F207808B8008619392C0830E3
:10086000CB006D20CA08031D372C06114814CA039B
:100870002D2C08308B0063008B01481C612C061561
:100880000130CB006D200230CB00CC010330CD0015
:100890000430CE000F200130CB006D200230CB00A1
:1008A000CC010330CD00CE010F200130CB006D20F4
:1008B0000230CB000B30CC003808CD003808CE0019
:1008C0000F20EC21861A7A2C0330CB000B30CC00A1
:1008D000CD01CE010F207808B800380F702C712C94
:1008E000B80A0230CB000B30CC003808CD003808F5
:1008F000CE000F20061A922C0330CB000B30CC0018
:10090000CD01CE010F207808B800B8080319892C52
:10091000B8030230CB000B30CC003808CD003808CB
:10092000CE000F20861B972C6E30F800AA2C061BD9
:100930009F2CA30803199F2C7030F800AA2C0130BB
:10094000C0070318C10A0319C20A0319C30AA72B57
:100950007330F8008A110A12162D84011F308305A6
:100960000F3083169F0083128610B8014428FF3091
:10097000CB006D20FF30CB006D20FF30CB006D2011
:10098000FF30CB006D209828272904220230CB00AD
:100990000B30CC002030CD002030CE000F200130B5
:1009A000A3007330BB00861F262D061F262DBD0118
:1009B0002308BC0063227808023C031DE32C0130AD
:1009C000A3007330BB00BD012308BC006322780B79
:1009D000182D0310FA01370CF900360CF800350C0D
:1009E000F7003007BC003108BD0078080318780F05
:1009F000BD073208BE0079080318790FBE07330817
:100A0000BF007A0803187A0FBF073308C300320803
:100A1000C2003108C1003008C0003F08C7003E08CE
:100A2000C6003D08C5003C08C400A52B7808BB00E3
:100A30003B086E3C0319202D3B08733C031D212D00
:100A4000A30A3B08703C031D262DA303D32C63008F
:02400E00FA3F77
:00000001FF
